:020000020000FC
:1000000012C050C08FC08EC08DC08CC077C031C0B0
:1000100089C088C087C086C085C084C083C082C0B4
:1000200081C080C07FC02FED2DBF2DE025BF20E413
:100030002BBF2AB128692AB929B12C6029B920E03F
:1000400020BF23BF22BF22E029BF8A9820E6A22F2B
:10005000BB2720E8C22FDD2713E51AD014E718D0FC
:1000600011E616D012E714D014E712D016D0789407
:10007000FFCF0FB70F930CB10D930D3019F00F9107
:100080000FBF189500E6A02FBB270F910FBF189543
:100090002BB12072E9F31CB908951AE0F9DF1DE0D5
:1000A000F7DF08953FB73F9332B73030F1F0333583
:1000B00048F000FC15C05395583010F0220C10C0C9
:1000C000110C0EC000FC02C003940AC0002453951A
:1000D000583018F0220C239403C0110C139400C064
:1000E000332732BF3F913FBF189555270024112475
:1000F000222433E033BF3F913FBF1895F8943FB7B8
:100100003F93332733BF32BF5D3040F0220C00FCF9
:100110002394112DBDDF122DBBDFBFDF3F913FBF09
:0601200078941895189573
:00000001FF
